:020000040800F2
:1000000000C0002099120008590D00085D0D00087D
:10001000610D0008650D0008690D00080000000072
:100020000000000000000000000000006D0D00084E
:10003000710D000800000000750D0008790D000822
:10004000E1120008E1120008E1120008E1120008C4
:10005000E1120008E1120008E1120008890D000811
:10006000E1120008E1120008E1120008910D0008F9
:100070009D0D0008A90D0008E1120008E11200081A
:10008000E1120008E1120008E1120008E112000884
:10009000E1120008E1120008E1120008E112000874
:1000A000E1120008E1120008E1120008E112000864
:1000B000B50D0008E1120008E1120008E112000885
:1000C000E1120008E1120008E1120008E112000844
:1000D000E1120008E1120008E1120008C10D000859
:1000E000E1120008E1120008E1120008E112000824
:1000F000E1120008E1120008E1120008E112000814
:10010000E1120008E1120008E1120008E112000803
:10011000E1120008E1120008E1120008E1120008F3
:10012000E1120008E1120008E1120008E1120008E3
:1001300000000000000000000000000000000000BF
:1001400000000000000000000000000000000000AF
:10015000000000000000000000000000000000009F
:10016000000000000000000000000000000000008F
:10017000000000000000000000000000000000007F
:10018000000000000000000000000000000000006F
:10019000000000000000000000000000000000005F
:1001A000000000000000000000000000000000004F
:1001B000000000000000000000000000000000003F
:1001C000000000000000000000000000000000002F
:1001D000000000000000000000000000000000001F
:0401E0005FF8E0F1F3
:1001E80010B5054C237833B9044B13B10448AFF369
:1001F80000800123237010BD1800002000000000BB
:10020800C44F000808B5034B1BB103490348AFF3BB
:10021800008008BD000000001C000020C44F00083A
:1002280070B54FF0FF0C4CF4E06C1CEA11541DBF84
:100238001CEA135594EA0C0F95EA0C0F00F0DEF84F
:100248002C4481EA030621EA4C5123EA4C5350EA34
:10025800013518BF52EA033541F4801143F4801385
:1002680038D0A0FB02CE4FF00005E1FB02E506F016
:100278000042E0FB03E54FF00006E1FB03569CF06B
:10028800000F18BF4EF0010EA4F1FF04B6F5007F71
:1002980064F5407404D25FEA4E0E6D4146EB0606E3
:1002A80042EAC62141EA55514FEAC52040EA5E506C
:1002B8004FEACE2EB4F1FD0C88BFBCF5E06F1ED816
:1002C800BEF1004F08BF5FEA500E50F1000041EB4D
:1002D800045170BD06F0004646EA010140EA0200FA
:1002E80081EA0301B4EB5C04C2BFD4EB0C0541EA1C
:1002F800045170BD41F480114FF0000E013C00F331
:10030800AB8014F1360FDEBF002001F0004170BD54
:10031800C4F10004203C35DA0C341BDC04F114046D
:10032800C4F1200500FA05F320FA04F001FA05F2F9
:1003380040EA020001F0004221F0004110EBD370C6
:1003480021FA04F642EB06015EEA430E08BF20EAF2
:10035800D37070BDC4F10C04C4F1200500FA04F395
:1003680020FA05F001FA04F240EA020001F0004127
:1003780010EBD37041F100015EEA430E08BF20EA9A
:10038800D37070BDC4F1200500FA05F24EEA020EE2
:1003980020FA04F301FA05F243EA020321FA04F011
:1003A80001F0004121FA04F220EA020000EBD370C8
:1003B8005EEA430E08BF20EAD37070BD94F0000FC8
:1003C8000FD101F00046400041EB010111F4801FFC
:1003D80008BF013CF7D041EA060195F0000F18BFAD
:1003E800704703F00046520043EB030313F4801FE9
:1003F80008BF013DF7D043EA0603704794EA0C0FA3
:100408000CEA135518BF95EA0C0F0CD050EA4106B8
:1004180018BF52EA4306D1D181EA030101F0004135
:100428004FF0000070BD50EA410606BF104619465D
:1004380052EA430619D094EA0C0F02D150EA013669
:1004480013D195EA0C0F05D152EA03361CBF1046AA
:1004580019460AD181EA030101F0004141F0FE4149
:1004680041F470014FF0000070BD41F0FE4141F4CD
:10047800780170BD81F0004102E000BF83F00043C5
:1004880030B54FEA41044FEA430594EA050F08BF27
:1004980090EA020F1FBF54EA000C55EA020C7FEAEB
:1004A800645C7FEA655C00F0E2804FEA5454D4EB68
:1004B8005555B8BF6D420CDD2C4480EA020281EA32
:1004C800030382EA000083EA010180EA020281EA6A
:1004D8000303362D88BF30BD11F0004F4FEA0131BC
:1004E8004FF4801C4CEA113102D0404261EB4101CB
:1004F80013F0004F4FEA03334CEA133302D0524251
:1005080063EB430394EA050F00F0A780A4F101040C
:10051800D5F1200E0DDB02FA0EFC22FA05F2801846
:1005280041F1000103FA0EF2801843FA05F359412C
:100538000EE0A5F120050EF1200E012A03FA0EFCAB
:1005480028BF4CF0020C43FA05F3C01851EBE371D5
:1005580001F0004507D54FF0000EDCF1000C7EEBF2
:1005680000006EEB0101B1F5801F1BD3B1F5001F30
:100578000CD349085FEA30004FEA3C0C04F101044F
:100588004FEA445212F5800F80F09A80BCF1004F78
:1005980008BF5FEA500C50F1000041EB045141EAFA
:1005A800050130BD5FEA4C0C404141EB0101013CC3
:1005B80028BFB1F5801FE9D291F0000F04BF0146B2
:1005C8000020B1FA81F308BF2033A3F10B03B3F184
:1005D80020020CDA0C3208DD02F1140CC2F10C0214
:1005E80001FA0CF021FA02F10CE002F11402D8BF72
:1005F800C2F1200C01FA02F120FA0CFCDCBF41EA3E
:100608000C019040E41AA2BF01EB0451294330BD0C
:100618006FEA04041F3C1CDA0C340EDC04F11404E9
:10062800C4F1200220FA04F001FA02F340EA0300C0
:1006380021FA04F345EA030130BDC4F10C04C4F106
:10064800200220FA02F001FA04F340EA03002946E6
:1006580030BD21FA04F0294630BD94F0000F83F430
:10066800801306BF81F480110134013D4EE77FEA13
:10067800645C18BF7FEA655C29D094EA050F08BF5F
:1006880090EA020F05D054EA000C04BF1946104640
:1006980030BD91EA030F1EBF0021002030BD5FEA84
:1006A800545C05D14000494128BF41F0004130BDAC
:1006B80014F580043CBF01F5801130BD01F0004500
:1006C80045F0FE4141F470014FF0000030BD7FEA73
:1006D800645C1ABF194610467FEA655C1CBF0B466E
:1006E800024650EA013406BF52EA033591EA030F85
:1006F80041F4002130BD00BF90F0000F04BF00217D
:10070800704730B54FF4806404F132044FF00005AF
:100718004FF0000150E700BF90F0000F04BF002128
:10072800704730B54FF4806404F1320410F000458E
:1007380048BF40424FF000013EE700BF42004FEA89
:10074800E2014FEA31014FEA02701FBF12F07F4306
:1007580093F07F4F81F06051704732F07F4208BFBD
:10076800704793F07F4F04BF41F40021704730B5C4
:100778004FF4607401F0004521F000411CE700BF10
:1007880050EA010208BF704730B54FF000050AE093
:1007980050EA010208BF704730B511F0004502D594
:1007A800404261EB41014FF4806404F132045FEA96
:1007B800915C3FF4D8AE4FF003025FEADC0C18BF3F
:1007C80003325FEADC0C18BF033202EBDC02C2F131
:1007D800200300FA03FC20FA02F001FA03FE40EAC3
:1007E8000E0021FA02F11444BDE600BF4FF0FF3CB1
:1007F80006E000BF4FF0010C02E000BF4FF0010C13
:100808004DF804CD4FEA410C7FEA6C5C4FEA430C8B
:1008180018BF7FEA6C5C1BD001B050EA410C0CBFDA
:1008280052EA430C91EA030F02BF90EA020F00203C
:10083800704710F1000F91EA030F58BF994208BFA3
:1008480090422CBFD8176FEAE37040F00100704760
:100858004FEA410C7FEA6C5C02D150EA013C07D1B7
:100868004FEA430C7FEA6C5CD6D152EA033CD3D002
:100878005DF8040B704700BF8446104662468C46FC
:100888001946634600E000BF01B5FFF7B7FF00282F
:1008980048BF10F1000F01BD4DF808EDFFF7F4FF58
:1008A8000CBF012000205DF808FB00BF4DF808EDE3
:1008B800FFF7EAFF34BF012000205DF808FB00BF06
:1008C8004DF808EDFFF7E0FF94BF012000205DF828
:1008D80008FB00BF4DF808EDFFF7CEFF94BF0120DD
:1008E80000205DF808FB00BF4DF808EDFFF7C4FFD6
:1008F80034BF012000205DF808FB00BF4FEA410229
:1009080012F5001215D211D56FF47873B3EB625259
:1009180012D94FEAC12343F0004343EA505311F080
:10092800004F23FA02F018BF404270474FF0000012
:10093800704750EA013005D111F0004008BF6FF050
:10094800004070474FF00000704700BF00234FF48D
:100958006021012230B51248124C85B0C0E901333C
:10096800CDE901330460009303730375C16102612B
:1009780000F00EFD60B90A240125072369460848DE
:10098800CDE90045029300F011FE20B905B030BD55
:1009980000F0BAF9EFE700F0B7F905B030BD00BFD5
:1009A800800000200024014070B50024204B02681C
:1009B80086B09A42CDE90244CDE9044401D006B09C
:1009C80070BD03F56C439A6902A942F400729A61FA
:1009D8009A69054602F400720092009A9A69154EC7
:1009E80042F010029A619B69012203F010030193FF
:1009F800032301981048CDE9022301F0E9FA0F49D1
:100A080080224FF48073C6E900144FF480613046A9
:100A1800C6E90644C6E90323B460716101F032F8FF
:100A280018B92E62756206B070BD00F06DF9F8E76E
:100A38000024014038000020001001400800024056
:100A4800002330B50D480E4A83B0CDE9003302606B
:100A580000F084FF58B900240025002269460748A1
:100A6800CDE9004500F0E0FF20B903B030BD00F04B
:100A78004BF9F0E700F048F903B030BDB0000020B2
:100A880000740040002330B5154A016887B09142D0
:100A9800CDE90233CDE9043301D007B030BD1024CD
:100AA800032503F1804303F50433DA690D4842F066
:100AB8000052DA61DA6902A902F000520092009A43
:100AC8009A6942F004029A619B69CDE9024503F0F4
:100AD80004030193019B01F07BFA07B030BD00BF0E
:100AE8000074004000080140134B00B5586983B0FA
:100AF80040F0010058615B69002203F00103022104
:100B080001930B20019B00F0C7FE0B2000F000FFB3
:100B1800002203210C2000F0BFFE0C2000F0F8FE9C
:100B28000D200022032100F0B7FE0D2003B05DF870
:100B380004EB00F0EDBE00BF00100240F0B5002449
:100B480089B0CDE90444CDE906443B4B01259A69B7
:100B58003A4F42F020029A619A69394E02F0200217
:100B68000092009A9A69384642F010029A619A698E
:100B78004FF4805102F010020192019A9A6942F0F2
:100B880004029A619A6902F004020292029A9A692E
:100B980042F008029A619B69224603F00803039316
:100BA800039B01F053FB2A4630464FF4004101F005
:100BB8004DFB0222234B304604A9CDE904230694B9
:100BC80001F006FA6C220023304604A9CDE904237B
:100BD800069401F0FDF94FF44872002304A91A485D
:100BE800CDE90423069401F0F3F9032200233846E3
:100BF80004A9CDE90423069401F0EAF94FF48053DF
:100C0800384604A90493CDE90554079501F0E0F9A5
:100C18004FF40043304604A90493CDE905540795E1
:100C280001F0D6F922462946072000F035FE0720B4
:100C380000F06EFE09B0F0BD00100240000C01404B
:100C480000080140000021100010014030B50023C9
:100C5800012401224FF4803597B0CDE910234FF4D9
:100C680000314FF45012CDE90C45CDE9023302248E
:100C7800CDE90433CDE90733CDE909330F93019367
:100C8800069312930B934FF480330CA8CDE91432DA
:100C98000E91139401F0F4FA08B172B6FEE7034618
:100CA8000F22CDE9024305934FF48063214601A842
:100CB8000493019201F0D2FC08B172B6FEE74FF43A
:100CC800004306A80694089301F0AAFD08B172B67D
:100CD800FEE717B030BD00BF08B500F023FBFFF7F3
:100CE800B5FFFFF72BFFFFF7FFFEFFF72FFEFFF71C
:100CF800A7FE00F06BF900F029FA00F0CFF900F038
:100D080095F803F03BFFFEE772B6FEE70E4B82B0A4
:100D18009A690E4942F001029A619A6902F0010249
:100D28000092009ADA6942F08052DA61DB6903F0D6
:100D380080530193019B4B6823F0E06343F00073F9
:100D48004B6002B0704700BF001002400000014035
:100D5800FEE700BFFEE700BFFEE700BFFEE700BFFB
:100D6800FEE700BF704700BF704700BF704700BF75
:100D780008B500F0E9FABDE8084003F0E5BF00BF98
:100D8800022001F071BA00BF014800F0CBBF00BFDC
:100D980038000020014800F0C5BF00BFE80100206E
:100DA800014800F0BFBF00BFA0010020014802F0C9
:100DB800EDB900BF0C01002010B5164C82B02046DA
:100DC80002F072FD23681B68DB0601D402B010BD77
:100DD800204602F097FB00212368019119680E4C08
:100DE80001915B6822780193019B42B14FF4007234
:100DF8000A49084802B0BDE8104002F04FBF084B4E
:100E080006491B6807485A685242D2B2227004F059
:100E1800C7F8EBE730020020B0090020B007002037
:100E2800A0010020B0030020704700BF30B50023A8
:100E38004FF0804541F2707442F20F7180221A48D7
:100E48008BB0C0E90054CDE90333CDE90533CDE9D2
:100E58000733C16000930293836003618261019349
:100E680001F0AAFDB0B90022002369460E48CDE979
:100E7800002302F035FAA0B90022002400250A4810
:100E880002A9CDE902450492069201F0A3FF20B918
:100E98000BB030BDFFF738FFE5E7FFF735FF0BB0C4
:100EA80030BDFFF731FFE7E70C010020104A036867
:100EB80082B0934210D00F4A934201D002B07047DB
:100EC8000D4BDA6942F00202DA61DB6903F00203D2
:100ED8000193019B02B07047074B9A6942F4006284
:100EE8009A619B6903F400630093009B02B070470A
:100EF800002C014000040040001002400368B3F1D8
:100F0800804F00D0704703F50433D96900B541F02C
:100F18000101D961DB6983B003F0010301931C204F
:100F280000220B21019B00F0B7FC1C2003B05DF8E8
:100F380004EB00F0EDBC00BF002370B51F49026848
:100F480086B08A42CDE90233CDE9043304D01C4B84
:100F58009A421BD006B070BD4FF480440225032688
:100F680003F1804303F504339A69164842F00802F6
:100F78009A619B6902A903F008030093CDE9024531
:100F8800009B059601F024F806B070BD8024022568
:100F9800032603F503339A690B4842F004029A6169
:100FA8009B6902A903F004030193CDE90245019B63
:100FB800059601F00DF806B070BD00BF002C014089
:100FC80000040040000C01400008014030B5002436
:100FD80093B0202221460AA8CDE90144CDE9034473
:100FE800CDE90544CDE90744009403F0ADFF3B2368
:100FF800284843604FF47A73C360274BC0E9044420
:1010080084608461036001F04DFD002831D1002225
:10101800002369461F48CDE9002302F061F9002842
:1010280034D160254FF4FA740023CDE9025400242A
:1010380000250422174802A9CDE906450493059323
:10104800089301F097FFF0B9002300244FF40055EE
:1010580010480AA9CDE90E45CDE90B330A930D9343
:10106800119302F077F938B90A48FFF765FF13B012
:1010780030BDFFF749FECAE7FFF746FE0548FFF710
:101088005BFF13B030BDFFF73FFEDDE7FFF73CFE27
:10109800C7E700BF58010020002C014000230220B0
:1010A80010214FF4FA62D0B5264C8AB0CDE903334B
:1010B800CDE90533CDE90733009302932361A3619A
:1010C8000193214BC4E901012046E260236001F04D
:1010D800E9FC28BB08211B4801F006FE40BB0022A2
:1010E800002369461748CDE9002302F0F9F828BB28
:1010F800042260264FF4FA770023124802A9CDE9AA
:1011080002670493069201F035FFA0B922680D48E2
:10111800936923F400639361FFF70EFF0AB0D0BD13
:10112800FFF7F2FD0821074801F0DEFD0028D6D0C0
:10113800FFF7EAFDD3E7FFF7E7FDE7E7FFF7E4FD91
:10114800D6E700BFC40000200004004000234FF48D
:10115800E1310C2210B50948094CC0E90113C0E976
:101168000333C0E905230460C36102F021F900B923
:1011780010BDBDE81040FFF7C7BD00BF300200201A
:101188000048004070B500243A4B026886B09A4285
:10119800CDE90244CDE9044401D006B070BD03F5A1
:1011A800E433DA69054642F48022DA61DA693248C2
:1011B80002F480220092009A9A69304E42F010029E
:1011C8009A619B694FF4806203F0100301930199BF
:1011D80003210223059102A9CDE9022300F0F8FEBC
:1011E8004FF400620023244802A9CDE902230494A5
:1011F80000F0EEFE224AB4605368346123F03003F5
:1012080043F0E06343F0100353601E4B102180222B
:1012180033604FF480533046C6E905447160F2608C
:10122800F36100F02FFCF8B900234FF480528021BD
:10123800154CAE63C4E90133C4E90433C4E906328A
:10124800124B20467562E160236000F01BFC70B908
:10125800002202212720EC63656200F01DFB272095
:1012680000F056FB06B070BDFFF74EFDDCE7FFF758
:101278004BFDEDE70048004000100140E801002068
:10128800000001401C000240A00100203000024084
:10129800FFF7CAFD0B480C490C4A002302E0D4585A
:1012A800C4500433C4188C42F9D3094A094C0023AA
:1012B80001E013600432A242FBD303F04DFEFFF7B6
:1012C8000BFD704700000020140000206850000843
:1012D80018000020CC0A0020FEE7000038B54FF4C3
:1012E8007A730D4A054611780C4AB3FBF1F312687C
:1012F800B2FBF3F000F01AFB08B90F2D01D9012059
:1013080038BD0446024629464FF0FF3000F0C4FAC3
:10131800034B20461D6038BD04000020000000205B
:1013280008000020074A08B51368032043F010039B
:10133800136000F09FFA0A20FFF7D0FFFFF7E6FCE2
:10134800002008BD00200240034A044B11681B78A6
:101358000B441360704700BF78020020040000208F
:10136800014B1868704700BF7802002038B5044662
:10137800FFF7F6FF631C054602D0044B1B781C449C
:10138800FFF7EEFF401BA042FAD338BD040000204F
:10139800002800F0968038B5836A0446002B72D086
:1013A80023689A68D1074CD4A26AD20605D5A36AE5
:1013B80043F01003A362012038BDA26A574822F403
:1013C800885222F0020242F002028342A262E169DC
:1013D800626870D0257B94F814C042EA45020A433B
:1013E800A168B1F5807F54D0A1F10100B0FA80F076
:1013F800BCF1010F4FEA50104FEA002064D05D683D
:1014080025F46945284358609D684548284010439D
:10141800986001294BD00020D96A21F4700101435A
:10142800D96299683F4B0B409A4267D0A36A23F070
:10143800120343F01003A362E36A43F00103E3627B
:10144800B9E79A6822F001029A60FFF789FF2368DA
:1014580005469A68D207A7D502E09A68D107A3D5AE
:10146800FFF77EFF401B02282368F6D99A68D00749
:10147800F3D5A36A43F01003A362E36A43F00103C0
:10148800E362A36A93E7C36280F82430FFF78CFA1B
:1014980086E7BCF1010F16D05868214920F469404D
:1014A80040F4807058609868014011439960206941
:1014B80001380005B0E7B1F5402F08BF4FF400210F
:1014C80088E70120704708460DB3A56A45F0200556
:1014D800A562E56A45F00105E5625D68B1F5807FC2
:1014E80025F4694540EA050058609D680C4800EA03
:1014F800050040EA020098608BD1D8E70020E0623E
:10150800A36A23F0030343F00103A36238BDA5696E
:10151800013D40EA453040F40060DEE7003C014010
:10152800FDF7E1FFFE0E1FFF704700BF436A9A6A8E
:1015380012F0500F0FD19A6A196842F4007210B570
:101548009A628A6802F46022B2F5602F06D01846C3
:10155800FFF7EAFF10BD1B6A1B6B18471A7B002AAE
:10156800F5D19A6A22F480729A629A6AD204EED409
:101578009A6A42F001029A62E9E700BF704700BF29
:1015880008B5406AFFF7FAFF08BD00BF704700BF03
:10159800406A08B5836A43F040038362C36A43F034
:1015A8000403C362FFF7F2FF08BD00BF002230B595
:1015B80083B0019290F82420012A66D003460120C6
:1015C80083F824004C681A68062C086804EB840C1D
:1015D8002FD90C2C4BD81F25146BACF1230C05FA12
:1015E8000CF500FA0CFE24EA050444EA0E04146320
:1015F8000928896800EB40042DD94FF0070C1E3CE0
:10160800A1400CFA04FCD46824EA0C042143A0F19C
:101618001004012CD16028D82C498A4238D00120E6
:101628009A6A42F020029A62002283F8242003B0CA
:1016380030BD4FF01F0E546BACF1050C00FA0CF5E1
:101648000EFA0CFC24EA0C042C430928546389681C
:1016580000EB4004D1D84FF0070C1069A1400CFAF8
:1016680004F420EA0400014311610020DCE71F258F
:10167800D46AACF1410C05FA0CF500FA0CFE24EA28
:10168800050444EA0E04D462B2E7022003B030BD78
:1016980091680902E9D49168102841F40001916029
:1016A800E3D10B4A0B491268A1FB0212920C02EB20
:1016B800820252000192019A002AD6D0019A013A78
:1016C8000192019A002AF9D1CFE700BF0024014016
:1016D8000000002083DE1B43002330B5026883B07E
:1016E80001939368D90727D41B4B04461B681B48F2
:1016F8009168A0FB030341F001019B0C91600193E9
:10170800019B2BB1019B013B0193019B002BF9D15C
:10171800FFF726FE236805469B68DA070CD4FFF717
:101728001FFE431B022B236803D99A6812F001029B
:1017380005D09B68DB07F2D5002003B030BD01203F
:10174800A36A84F8242043F01003A362E36A0343E6
:10175800E36203B030BD00BF0000002083DE1B43FE
:10176800F8B504463E4D00680F46A842164659D0C3
:101778003C4B984256D094F82430012B5FD001237B
:10178800204684F82430FFF7A7FF0546002851D1EA
:10179800A06A2168334B20F4706020F0010040F407
:1017A80080709942A0624DD0A36A23F48013A3628B
:1017B8004B685A0505D5A36A23F4405343F4805374
:1017C800A362A36A002013F4805318BFE36A84F865
:1017D800240018BF23F00603E36233466FF00206C5
:1017E800206A3A46204F4C318762204FC762204F0B
:1017F800076341F84C6C51F8446C46F4807641F824
:10180800446C00F08BF9236828469A6802F4602239
:10181800B2F5602F9A680CBF42F4A00242F480121D
:101828009A60F8BD0E4B5B6813F4702FA3D00125A6
:101838002846F8BD002384F824302846F8BD022540
:101848002846F8BDA3F580635A6812F4702FABD010
:10185800A26A42F48012A2625B685B05B1D5AAE76E
:1018680000240140002801403515000889150008AA
:10187800991500084FF6FF0C06490302CA6803F4DD
:10188800E06302EA0C02134343F0BF6343F40033FE
:10189800CB60704700ED00E01B4B00B5DB68C3F37D
:1018A8000223C3F1070EBEF1040F03F1040C28BF95
:1018B8004FF0040EBCF1060F1CD9A3F1030C4FF036
:1018C800FF3303FA0CF322EA03024FF0FF3303FA63
:1018D8000EF321EA030303FA0CF313431B01002858
:1018E800DBB20ADB00F1604000F5614080F80033AC
:1018F8005DF804FB00229446E7E7044A00F00F0075
:10190800024413765DF804FB00ED00E0FCEC00E017
:10191800002807DB012300F01F01034A40098B4020
:1019280042F82030704700BF00E100E00138B0F114
:10193800807F01D3012070474FF0E0234FF0F00C77
:101948000022072110B4044C586184F823C01046C3
:101958009A6110BC1961704700ED00E088B110B5BC
:101968000379044603F0FF023BB100230221012260
:10197800217123612271184610BD4271FFF782F868
:10198800F3E70120704700BF68B342790346012A94
:101998002BD010B40224012200681C71046801F0E5
:1019A800100C02FA0CF22243026079B9026802F0C4
:1019B8003C023C2A03D1426842F001024260002204
:1019C80001215A711971104610BC70473C220168F8
:1019D80002FA0CF201F470119142F0D1426842F01F
:1019E80002024260EBE7012070470220704700BF07
:1019F80010B4002483B0019488B10068019049B103
:101A0800019914310A4401920020019A136003B02D
:101A180010BC7047019908310A440192F4E701208B
:101A280003B010BC704700BF38B331B303464079E8
:101A3800012824D0022070B54FF0C00C40F6FE7685
:101A48004FF0000E012518711C68D1E9000102F061
:101A58001002014396400CFA02FC01FA02F22168D6
:101A6800704621EA06010A432260226822EA0C0233
:101A780022601D7183F805E070BD012070470220C7
:101A8800704700BF00283AD001681E4A03469142B9
:101A980010B42BD91C4A1D480A44A0FB02021C4C56
:101AA80012099200C3E90F42D3E901242243DC68FA
:101AB800022022431C694FF0010C22435C6983F821
:101AC800210022439C6908682243DC6920F47F5086
:101AD8002243002420F0300002430A609C6383F80C
:101AE800204083F821C0204610BC7047094A0748A7
:101AF8000A44A0FB02021209074C9200D2E7012017
:101B0800704700BF07040240F8FBFDBFCDCCCCCC2A
:101B180000040240F8FFFDBF0000024070B490F8D6
:101B28002040012C0BD0012590F8214080F820504E
:101B3800AC425FFA84FC05D0002380F820300220F4
:101B480070BC7047022480F8214000248463046834
:101B5800056C26680CFA05F526F001062660C66BAA
:101B6800756063604368102BC36A0BBFA260A160F5
:101B7800E160E26053B1236843F00E0323602368F9
:101B8800002043F00103236070BC7047236823F0F2
:101B980004032360236843F00A032360EFE700BFD0
:101BA80090F821200346022A06D004229A630022D4
:101BB800012083F8202070474FF0010C1A6800209C
:101BC800116821F00E011160116821F00101116006
:101BD800D3E90F120CFA02F24A60002283F821C0FE
:101BE80083F82020704700BF08B590F821200346ED
:101BF800022A03D0042201209A6308BD02684548DE
:101C08001168824221F00E011160116821F0010172
:101C18001160414924D98A4256D014318A425FD092
:101C280014318A425ED014318A4254D014318A4227
:101C380061D014318A4264D0824268D001F567715C
:101C48008A4241D014318A424AD014318A4249D05A
:101C580014318A4214BF4FF480324FF4805234E07A
:101C68008A4222D014318A4238D014318A423CD078
:101C780014318A422CD014318A4239D014318A4224
:101C88003CD0824240D001F567718A420DD01431B0
:101C98008A4223D014318A4227D014318A4214BF91
:101CA8004FF480324FF4805200E001221B494A6011
:101CB800012000215A6B83F8210083F820100AB113
:101CC80018469047002008BD012215494A60EFE7F1
:101CD8004FF48052EAE74FF48052F6E71022E5E726
:101CE8001022F2E74FF48072EFE74FF48072DDE7DD
:101CF8004FF48032DAE74FF48032E6E74FF480128F
:101D0800D4E74FF48012E0E74FF08072CEE74FF04F
:101D18008072DAE7800002400800024000000240BA
:101D280000040240042270B4C66B016C3468036876
:101D38008A4022421D6843D06A0741D51A68910635
:101D480003D41A6822F004021A609C4A9C49934200
:101D580040F293808B4200F0F18014318B4200F006
:101D6800F58014318B4200F0E48014318B4200F08E
:101D7800F88014318B4200F0008114318B4200F05E
:101D88000581934200F00E8102F56272934200F0E1
:101D9800D5801432934200F0D9801432934200F077
:101DA800C8801432934214BF4FF480234FF4804309
:101DB800844A5360C36A002B40F0B28070BC7047FD
:101DC80002228A4022423FD0AA073DD51A689106CE
:101DD80006D401211A6822F00A021A6080F821103C
:101DE800764A774993426FD98B4200F0A980143123
:101DF8008B4200F0998014318B4200F0A980143195
:101E08008B4200F0B18014318B4200F0BC80143159
:101E18008B4200F0C480934200F0CD8002F56272DC
:101E2800934200F08D80143293427DD01432934255
:101E380000F08E801432934214BF4FF400324FF4F6
:101E48000052604B5A6064E008228A402242B5D0B2
:101E58002A07B3D51A68002422F00E021A6001235B
:101E6800026B03FA01F17160836380F8204080F807
:101E78002130002AA2D070BC10478B425CD01431AC
:101E88008B4261D014318B4250D014318B4265D0D3
:101E980014318B426ED014318B427AD0934200F0C9
:101EA8008480494A934247D0143293424CD014322A
:101EB80093423BD01432934214BF4FF480234FF423
:101EC8008043424A536075E78B423BD014318B42C2
:101ED80028D014318B423ED014318B4247D0143174
:101EE8008B424DD014318B4256D0934260D0364A43
:101EF800934227D01432934214D0143293422AD0FA
:101F08001432934214BF4FF400324FF400522F4B57
:101F18005A600022836A80F82020002B3FF44EAFDD
:101F280070BC18472022F2E720228AE74FF480632A
:101F3800C7E74FF480633BE70423C2E7042337E78E
:101F480002227EE70222E2E74023BAE740232FE796
:101F58004FF4007275E74FF40072D8E74FF48043EE
:101F6800AFE74FF4804323E74FF4005269E74FF49B
:101F78000052CCE74FF48023A3E74FF4802317E700
:101F88004FF40032C3E74FF400325AE74FF48003AE
:101F98000EE74FF4800394E74FF40012B7E74FF4CD
:101FA80000124EE74FF0806302E74FF0806388E746
:101FB8004FF00072ABE74FF0007242E7800002403A
:101FC80008000240000402400804024000000240E9
:101FD8002DE9F04F0D6883B0002D00F0CE8000226F
:101FE8008C4E92461346DFF830828C4F06E0013360
:101FF80035FA03F402F1040200F0BF8001249C408A
:1020080034EA050E04EA050CF1D14D68122D00F2F0
:10201800B780122D1AD8DFE805F0BED0CCD7191931
:102028001919191919191919191919C8D300DFF823
:10203800F0E1754500F0AF800EF5702E754500F0A3
:10204800AA80AEF5801E754500F0A580BCF1FF0F93
:102058009CBF864693464FF00F0584BF00F1040EDF
:10206800A2F1200BDEF800400AFA0BF905FA0BFB87
:1020780024EA0B0444EA0904CEF800404C6814F042
:10208800805F00F09080D6F818E003F003094EF066
:10209800010EC6F818E0D6F818E04FEA89090EF0E4
:1020A800010ECDF804E0DDF804E023F0030E0EF194
:1020B800804E0EF5803EDEF808B005FA09F52BEAE9
:1020C8000505DFF860B158451ED00BF5806B584503
:1020D80000F08480DFF850B1584578D0DFF84CB173
:1020E800584500F08980DFF848B1584500F08B80EA
:1020F800DFF840B158450CBF4FF0050B4FF0060B09
:102108000BFA09F945EA0905CEF80850DFF828E185
:1021180014F4801FDEF8085014BF45EA0C0525EAC0
:102128000C05CEF80850DFF810E114F4001FDEF8B3
:102138000C5014BF45EA0C0525EA0C05CEF80C50E6
:10214800DFF8F4E014F4003FDEF8045014BF45EA69
:102158000C0525EA0C05CEF80450374D14F4803FE1
:102168002C681DD044EA0C042C600D68013335FA44
:1021780003F402F104027FF441AF03B0BDE8F08F2D
:10218800454508D07FF653AFBD4204D0DFF8ACE038
:1021980075457FF45BAF8D683DBB4FF0040A55E78A
:1021A80024EA0C042C600D6821E7CC6804F1040AC9
:1021B8004CE7CC6804F1080A48E7D1F80CA045E7D9
:1021C800CC6804F10C0A41E74FF0000A3EE74FF0F3
:1021D800020B0BFA09F945EA090595E74FF0010BDF
:1021E8000BFA09F945EA09058EE7012D4FF0080AAF
:1021F8000CBF0461446129E74FF0030B0BFA09F99E
:1022080045EA090580E74FF0040B0BFA09F945EA9E
:10221800090579E700100240000022100000311083
:102228000000121000080140001001400014014095
:1022380000180140001C0140000401400000321059
:102248008368194214BF01200020704702B90904AD
:1022580001617047C36801EA030221EA030141EA08
:1022680002410161704700BF044A5169014200D12F
:10227800704708B5506102F0CBF808BD0004014072
:10228800002800F0E4812DE9F04103680446DD07E9
:1022980082B035D599494A6802F00C02042A00F048
:1022A800ED804A6802F00C02082A00F0E3806368B7
:1022B800B3F5803F10D0002B00F00A81B3F5A02FB2
:1022C80000F080818D4B1A6822F480321A601A68F7
:1022D80022F480221A6004E0884A136843F48033A9
:1022E8001360FFF73DF8854E054605E0FFF738F81F
:1022F800401B642800F2E88033689A03F6D5236807
:102308009F0728D57D4A516811F00C0F00F0968080
:10231800516801F00C01082900F08C802369002B1A
:1023280000F016810122764B744E1A60FFF718F8F8
:10233800054605E0FFF714F8401B022800F2C480A8
:1023480033689807F6D53368626923F0F80343EADF
:10235800C203336023681A0729D45D074BD5674B3E
:10236800DA69D00000F184800125DA6942F08052F0
:10237800DA61DB6903F080530093009B614E336898
:10238800D90540F19180E368012B00F0F280002B21
:1023980000F0BE80052B594B1A6A00F0208122F00C
:1023A80001021A621A6A22F004021A62E6E0A369BC
:1023B800002B4CD00122524B504EC3F88024FEF71C
:1023C800CFFF054604E0FEF7CBFF401B02287BD871
:1023D800736A9B07F7D54C4B4C4A1B68A2FB032337
:1023E8005B0A019300BF019B5A1E0192002BF9D191
:1023F80023685D07B3D4E369C3B1404D6A6802F04E
:102408000C02082A00F0CD800022022B3C4B1A66F1
:1024180000F0ED80FEF7A4FF044604E0FEF7A0FFFD
:10242800001B022850D82B689B01F7D4002002B06B
:10243800BDE8F0815268D6033FF570AF2F4A1268A5
:10244800950725D52269012A22D00120EFE72C4AD9
:102458002A4EC2F88034FEF783FF054604E0FEF7F3
:102468007FFF401B02282FD8736A9F07F7D4BFE766
:10247800002583E74A68D0037FF519AF1F4A126821
:1024880091037FF53DAF6268002A7FF439AFDCE73E
:102498001A4960690A6822F0F80242EAC0020A6032
:1024A8001A077FF55AAF82E7336843F480733360C5
:1024B800FEF756FF07463368DA053FF564AFFEF7C7
:1024C8004FFFC01B6428F6D9032002B0BDE8F08195
:1024D8000A4D2B6823F480332B602B6823F4802368
:1024E8002B60FEF73DFF064604E0FEF739FF801B30
:1024F8006428E9D82B689B03F7D400E70010024052
:10250800000042420070004000000020D34D6210DD
:10251800504E41F28838336A23F001033362336A3C
:1025280023F004033362FEF71BFF074604E0FEF7BF
:1025380017FFC01B4045C7D8336A9807F7D4002D4A
:102548003FF459AF434AD36923F08053D36152E72C
:10255800414A404E1360FEF703FF054604E0FEF7CC
:10256800FFFE401B0228AFD833689907F7D42368C9
:10257800F1E6384A136A43F001031362FEF7F0FEEE
:1025880041F288380646334F04E0FEF7E9FE801B27
:10259800404599D83B6A9B07F7D5002D3FF42BAFF0
:1025A800D0E7012B3FF451AF6B68226A03F4803106
:1025B80091427FF44AAF606A03F47013181A18BF87
:1025C800012034E703F18043A3F53C331A6842F451
:1025D80080221A601A6842F480321A6081E642F05A
:1025E80004021A621A6A42F001021A62C6E7FEF78A
:1025F800B7FE064605E0FEF7B3FE801B02283FF64D
:1026080063AF2B689901F6D4236AB3F5803F05D1EF
:102618006A68A16822F400320A436A6001200D4DFD
:10262800616A6A680B4322F474120B4913436B60A6
:102638000866FEF795FE044605E0FEF791FE001BCE
:1026480002283FF641AF2B689A01F6D5EEE6012045
:10265800704700BF0010024000004242002800F00E
:10266800A180564A2DE9F0411368044603F0070398
:102678008B420D460CD2136823F007030B431360FB
:10268800136803F007038B4202D00120BDE8F081F4
:1026980023689E0714D5580704D549494A6842F467
:1026A800E0624A60190704D545494A6842F4605215
:1026B8004A604349A0684A6822F0F00202434A602F
:1026C800DA0720D562683E4B012A1B686CD0022AC3
:1026D80065D09E07D9D53A4E41F28838736823F001
:1026E800030313437360FEF73BFE074604E0FEF75F
:1026F80037FEC01B40455AD87368626803F00C0364
:10270800B3EB820FF3D12D4A136803F00703AB42F2
:1027180009D9136823F007032B431360136803F0E8
:102728000703AB42B1D12368580706D52449E068AE
:102738004A6822F4E06202434A60190707D5204A32
:102748002169536823F4605343EAC10353601C4969
:102758004A6802F00C03082B10D01A4B184A1A4882
:1027680052681A49C2F30312805C194AC3400868C8
:102778001360FEF7B3FD0020BDE8F0811548C2F3F1
:102788008343D203C35C14D50E484A6800FB03F3A5
:102798001149C2F340428A5CB3FBF2F3DEE79F01C2
:1027A80099D472E7012070479B0394D46DE7032006
:1027B8006CE70A4A02FB03F3D0E700BF002002409F
:1027C8000010024000127A00E44F000808000020C0
:1027D80000000020F84F0008F44F000800093D00F1
:1027E800044B054A5B680549C3F30223CB5C1068B8
:1027F800D84070470010024000000020DC4F00085D
:10280800044B054A5B680549C3F3C223CB5C1068D7
:10281800D84070470010024000000020DC4F00083C
:102828002DE9F04103680446D80782B02CD5394B0E
:10283800DA69D1003FD5384D00262B68DA0548D52E
:10284800344D61682B6A13F4407311D001F440725F
:102858009A420DD0002001272B6A304A23F4407198
:10286800C2F84074C2F84004D807296244D46168A9
:10287800284A136A23F440730B4313621EB1D369C9
:1028880023F08053D36123689A0706D52149A068AD
:102898004A6822F4404202434A60DB0603D400201F
:1028A80002B0BDE8F0811B4A6169536823F48003D4
:1028B8000B435360F3E7DA69174D42F08052DA614F
:1028C800DB69012603F080530193019B2B68DA052D
:1028D800B6D42B6843F480732B60FEF741FD07469E
:1028E8002B68DB05ACD4FEF73BFDC31B642BF7D983
:1028F800032002B0BDE8F081FEF732FD41F28838CE
:1029080007462B6A9907B2D4FEF72AFDC01B40453B
:10291800F7D9EDE700100240007000400000424285
:1029280090F83D30012B27D10222036880F83D2022
:10293800DA68124942F001028B42DA6011D0104A7B
:1029480093420ED0B3F1804F0BD0A2F59832934248
:1029580007D002F58062934203D002F58062934269
:1029680004D19A6802F00702062A03D01A6842F0D6
:1029780001021A600020704701207047002C0140B6
:102988000034014041F2111C02680346D16821F06D
:102998000101D160116A11EA0C0F08D140F24441DB
:1029A800106A084203D1116821F001011160012267
:1029B800002083F83D20704700286ED038B590F885
:1029C8003D30044603F0FF02002B61D00223226849
:1029D800334984F83D308A4213681CD001F5006100
:1029E8008A4218D0B2F1804F40D0A1F598318A427E
:1029F8003CD001F580618A4238D001F580618A4275
:102A080034D0A5696168E06823F080032B43136024
:102A1800D062916212E0A06823F070032169034339
:102A280023F440730B43A16923F080030B43136025
:102A3800E368D36263689362636913630123536134
:102A480084F8463084F83E3084F83F3084F84030CB
:102A580084F8413084F8423084F8433084F84430B4
:102A680084F8453084F83D30002038BDA16823F053
:102A7800700320690B4323F44073A169034323F0D7
:102A88008003E0680B4361681360D0629162D5E708
:102A980080F83C20FEF732FA98E70120704700BF23
:102AA800002C014000286ED038B590F83D3004461F
:102AB80003F0FF02002B61D002232268334984F817
:102AC8003D308A4213681CD001F500618A4218D053
:102AD800B2F1804F40D0A1F598318A423CD001F53F
:102AE80080618A4238D001F580618A4234D0A56974
:102AF8006168E06823F080032B431360D062916221
:102B080012E0A06823F070032169034323F44073A3
:102B18000B43A16923F080030B431360E368D3627E
:102B280063689362636913630123536184F84630D1
:102B380084F83E3084F83F3084F8403084F84130DF
:102B480084F8423084F8433084F8443084F84530BF
:102B580084F83D30002038BDA16823F07003206957
:102B68000B4323F44073A169034323F08003E06817
:102B78000B4361681360D0629162D5E780F83C200E
:102B8800FEF794F998E70120704700BF002C014038
:102B980099BB90F83E30012B3BD1022380F83E30A0
:102BA8000122036801F01F01186A8A4020EA020026
:102BB80010B41862196A224C0A43A3421A622AD036
:102BC800204A934227D0B3F1804F0AD01E4A93423D
:102BD80007D002F58062934203D002F580629342E7
:102BE80004D19A6802F00702062A03D01A6842F054
:102BF80001021A60002010BC7047042910D008296F
:102C080016D090F84130012B03D1022380F84130CF
:102C1800C6E7012070475A6C42F400425A64E0E764
:102C280090F83F30012BF4D1022380F83F30B7E70A
:102C380090F84030012BECD1022380F84030AFE708
:102C4800002C0140003401400004004001220368C8
:102C580001F01F0C02FA0CFC1A6A10B422EA0C02EA
:102C68001A621E4C1A6AA3421A6213D01C4A934273
:102C780010D041F211121C6A144204D140F24442AD
:102C88001C6A144220D0012399B980F83E3010BC48
:102C98000020704741F211121C6A1442E9D140F237
:102CA80044421C6A1442E4D15A6C22F400425A6429
:102CB800DFE704290DD008290CBF80F8403080F8E0
:102CC800413010BC002070471A6822F001021A60D7
:102CD800D9E780F83F3010BC00207047002C014035
:102CE80000340140704700BF00286ED038B590F816
:102CF8003D3004460D4603F0FF02002B60D002224F
:102D08002368334984F83D208B421A681CD001F5AA
:102D180000618B4218D0B3F1804F3FD0A1F59831B4
:102D28008B423BD001F580618B4237D001F5806141
:102D38008B4233D0A06922F0800261680243E068C8
:102D48001A60D862996212E0A16822F070020A4300
:102D5800216922F440720A43A16922F080020A43E1
:102D68001A60E268DA6262689A6262691A6301222A
:102D78005A611968002021F008011960196829436F
:102D8800196084F8462084F83E2084F83F2084F8AF
:102D9800422084F8432084F83D2038BDA16822F001
:102DA80070020A43216922F440720A43A16922F0A1
:102DB80080020A43E1681A606268D9629A62D6E7BB
:102DC80080F83C20FFF78EFF99E70120704700BF8D
:102DD800002C014090F83C30012B00F09180844693
:102DE80030B50C2A08D8DFE802F0310707074E078C
:102DF80007076D0707070C0000238CF83C300120FB
:102E080030BD03680D681A6A186A22F4005220F46B
:102E1800805018625C68D86920F4E64040EA0520D2
:102E28008D6842EA0532524DAB4200F08A8005F5C2
:102E38000065AB4200F0858049685C60D861196420
:102E48001A6200238CF83C30002030BD03680D68FE
:102E58001A6A186A22F0020220F0010018625C68FF
:102E6800986920F0730028438D682A43404DAB428F
:102E780048D005F50065AB4244D049685C6098616C
:102E880059631A62DDE703680D681A6A186A22F046
:102E9800200220F0100018625C68986920F4E6406F
:102EA80040EA05208D6842EA0512314DAB4238D020
:102EB80005F50065AB4234D049685C609861996358
:102EC8001A62BEE703680D681A6A186A22F400726B
:102ED80020F4807018625C68D86920F07300284379
:102EE8008D6842EA0522224DAB4230D005F50065D7
:102EF800AB422CD049685C60D861D9631A62A0E7FC
:102F080002207047CD6822F008022A4324F4407456
:102F1800D1E905E54EEA050E22F004024EEA040462
:102F2800ABE7CD6822F0800242EA051224F440643F
:102F3800D1E905E54EEA050E22F0400244EA8E0486
:102F4800BAE74D6924F4804444EA851474E7CD68EF
:102F580022F4006242EA052224F44054D1E905E54E
:102F68004EEA050E22F4806244EA0E14C2E700BF5E
:102F7800002C014090F83C30012B00F0C680012362
:102F880030B5844680F83C300C2A08D8DFE802F0D7
:102F98003E07070767070707930707070C00002383
:102FA8008CF83C30012030BD03680D681A6A186A35
:102FB80022F4005220F4805018625C68D86920F42A
:102FC800E64040EA05208D6842EA05326A4DAB4288
:102FD80000F0BC8005F50065AB4200F0B7805C608E
:102FE800D8614868096918641A62DA6942F40062AB
:102FF800DA61DA6922F48062DA61DA6942EA012286
:10300800DA6100238CF83C30002030BD03680D687D
:103018001A6A186A22F0020220F0010018625C683D
:10302800986920F0730028438D682A43524DAB42BB
:103038006DD005F50065AB4269D05C609861486861
:10304800096958631A629A6942F008029A619A6992
:1030580022F004029A619A690A439A61D1E70368E7
:103068000D681A6A186A22F0200220F0100018620F
:103078005C68986920F4E64040EA05208D6842EAD9
:1030880005123D4DAB4251D005F50065AB424DD020
:103098005C6098614868096998631A629A6942F4A1
:1030A80000629A619A6922F480629A619A6942EA96
:1030B80001229A61A5E703680D681A6A186A22F462
:1030C800007220F4807018625C68D86920F0730080
:1030D80028438D6842EA0522274DAB423CD005F5CE
:1030E8000065AB4238D05C60D86148680969D8632C
:1030F8001A62DA6942F00802DA61DA6922F0040237
:10310800DA61DA690A43DA617BE702207047CD6841
:1031180022F008022A4324F44074D1E905E54EEA76
:10312800050E22F004024EEA040486E7CD6822F078
:10313800800242EA051224F44064D1E905E54EEA2A
:10314800050E22F0400244EA8E04A1E74D6924F4FA
:10315800804444EA851442E7CD6822F4006242EADA
:10316800052224F44054D1E905E54EEA050E22F47F
:10317800806244EA0E14B6E7002C0140704700BF95
:10318800704700BF704700BF704700BF036810B5A5
:103198001A690446910702D5DA6892075FD41A695A
:1031A800500702D5DA68510746D41A69120702D5C2
:1031B800DA6810072ED41A69D20602D5DA68D00662
:1031C80018D41A69D10702D5DA68D2075DD41A690A
:1031D800100602D5DA6811065FD41A69520602D5BC
:1031E800DA68500661D41A69910602D5DA6892063F
:1031F80043D410BD6FF01001082219612277DB69F2
:10320800204613F4407F64D0FFF7BAFF00222368FA
:103218002277D6E76FF00801042219612277DB696B
:103228002046990752D1FFF7A9FF2046FFF7AAFFCA
:10323800002223682277BEE76FF004010222196199
:1032480022779B69204613F4407F3CD1FFF796FF15
:103258002046FFF797FF002223682277A5E76FF043
:1032680002010122196102779B699B0725D0FFF7AC
:1032780087FF00222368227791E76FF0200220461B
:10328800BDE810401A6100F08FB86FF001022046C7
:103298001A6101F08BFB236899E76FF080022046E2
:1032A8001A6100F083F8236897E76FF04002204620
:1032B8001A61FFF769FF236895E7FFF75FFF20466C
:1032C800FFF760FFD5E7FFF75BFFC4E7FFF758FF9D
:1032D800AEE7FFF753FF2046FFF754FF96E700BF1E
:1032E80090F83C20012A2FD0034602201A6830B4F7
:1032F80083F83D0050680C68144D20F0700020439E
:10330800AA429468506011D0114882420ED0B2F19E
:10331800804F0BD0A0F59830824207D000F580602E
:10332800824203D000F58060824204D1496824F0CB
:1033380080040C4394600022012183F83C2083F828
:103348003D10104630BC704702207047002C0140E9
:103358000034014090F83C30012B23D00246D1E9DB
:1033680002034FF0000C23F440730343486823F42E
:1033780080630343086823F400630343086923F464
:10338800805310B403434C6923F40053C8692343A2
:10339800116823F4804303434B6482F83CC06046C1
:1033A80010BC704702207047704700BF704700BFCD
:1033B800002865D070B590F84130044603F0FF024C
:1033C800002B55D0D4E902262421236884F8411023
:1033D800D968206921F40051A56902436069D96060
:1033E8001969024321F4405131431961D9682548CC
:1033F80021F4B05121F00C010A43DA605A69834282
:1034080022F4407242EA05025A6136D0FFF7E8F921
:10341800626800EB8003920003EB8303B3FBF2F3D3
:103428004FF0640E00254FF0200C17482168A0FBD0
:10343800036252090EFB12331B013233A0FB030354
:10344800120102EB53128A600B69284623F4904359
:103458000B614B6923F02A034B61CB6843F400539B
:10346800CB60656484F841C084F842C0656370BD70
:1034780080F84020FDF786FEA4E7FFF7C1F9C7E70B
:1034880001207047003801401F85EB51F8B504460C
:1034980090F84100202803D101B11AB90120F8BDE4
:1034A8000220F8BD00254FF0210EE284A2841346C5
:1034B800A06B2268DFF840C0104F114E656421628E
:1034C80084F841E00432C0E90AC7C0E90C65FEF798
:1034D80025FB6FF040032268136002F1140353E8E0
:1034E800003F43F0800302F1140040E80031002956
:1034F800F3D10020F8BD00BF01360008513600089E
:103508006936000810B503680446596990F84120E7
:10351800212A06D0596994F84220222A28D000206E
:1035280010BD0906F6D503F1140252E8002F22F067
:10353800800203F1140040E800210029F3D1A06BB8
:1035480010B1FEF72DFB236803F10C0252E8002F9F
:1035580022F0C00203F10C0040E800210029F3D159
:10356800202284F84120596994F84220222AD6D191
:103578004A06D4D503F1140252E8002F22F0400283
:1035880003F1140040E800210029F3D1E06B10B1E9
:10359800FEF706FB236803F10C0252E8002F22F421
:1035A800907203F10C0040E800210029F3D103F1E7
:1035B800140252E8002F22F0010203F1140040E83F
:1035C80000210029F3D1226B012A06D020220023F2
:1035D80084F842200020236310BD03F10C0252E856
:1035E800002F22F0100203F10C0040E8002100290E
:1035F800F3D1EBE7704700BF08B50368406A1B6862
:1036080013F020031AD10268C38402F1140353E8AB
:10361800003F23F0800302F1140040E80031002944
:10362800F3D102F10C0353E8003F43F0400302F1E9
:103638000C0040E800310029F3D108BDFFF7DAFF9C
:1036480008BD00BF704700BF08B5406AFFF7FAFF22
:1036580008BD00BF704700BF704700BF704700BF7C
:1036680008B5406A0368596990F84120212A0BD0AF
:10367800596990F84220222A1ED0436C43F0100367
:103688004364FFF7EBFF08BD0906F1D50022C284A9
:1036980003F10C0252E8002F22F0C00203F10C0CD7
:1036A8004CE800210029F3D1202280F841205969F3
:1036B80090F84220222AE0D14A06DED50022C285AF
:1036C80003F10C0252E8002F22F4907203F10C0C63
:1036D8004CE800210029F3D103F1140252E8002F2D
:1036E80022F0010203F1140C4CE800210029F3D167
:1036F800026B012A05D02022002380F842200363B0
:10370800BBE703F10C0252E8002F22F0100203F18C
:103718000C0C4CE800210029F3D1ECE708B5002394
:10372800406AC385C384FFF799FF08BD704700BF8F
:1037380008B50123406A4363036B012B02D0FFF7EE
:103748008BFF08BD818D4908FFF7F0FF08BD00BF5A
:1037580008B50368406A1A6812F020022BD1036882
:10376800C28503F10C0252E8002F22F4807203F1A3
:103778000C0C4CE800210029F3D103F1140252E8A3
:10378800002F22F0010203F1140C4CE8002100295B
:10379800F3D103F1140252E8002F22F0400203F1A2
:1037A800140C4CE800210029F3D1202280F8422093
:1037B800026B012A07D000234363036B012B0FD050
:1037C800FFF748FF08BD03F10C0252E8002F22F072
:1037D800100203F10C0C4CE800210029F3D1EAE7B0
:1037E800818DFFF7A3FF08BD83680168B3F5805F8B
:1037F800826A42D0002B39D04B6803F07F031370E4
:10380800826A0132C38D8262013B9BB2C385002B61
:1038180032D14FF0200C026800B5D16883B021F096
:103828002001D160D16821F48071D160516921F003
:103838000101516180F842C04363016B012925D120
:10384800036302F10C0353E8003F23F0100302F175
:103858000C0C4CE800310029F3D11368DB061AD4AC
:10386800818DFFF763FF03B05DF804FB0369002B4C
:10387800C2D14B68DBB2C2E770470369002BF8D1AD
:103888004B68C3F3080322F8023BBBE7FFF7E2FEED
:1038980003B05DF804FB0023019313680193536898
:1038A8000193019BDCE700BF30B5036804461A6842
:1038B80083B012F00F0FDD6859696FD1910602D5F8
:1038C800A90600F1A080216B01290BD0100602D5B2
:1038D800290600F1A280520602D5680600F1BC80D4
:1038E80003B030BDD006F1D5E906EFD5002201922C
:1038F8001A6801925A680192019A5A69550640F16C
:103908003581E06B0268526892B2002AE8D0A18D36
:103918009142E5D9E2858269202A36D003F10C026A
:1039280052E8002F22F4807203F10C0545E80021CB
:103938000029F3D103F1140252E8002F22F001020A
:1039480003F1140545E800210029F3D103F114021D
:1039580052E8002F22F0400203F1140545E8002147
:103968000029F3D1202284F84220216303F10C02BC
:1039780052E8002F22F0100203F10C0545E800215F
:103988000029F3D1FEF70CF9A18D02236363E38DBF
:103998002046C91A89B2FFF7C9FEA1E711F0010153
:1039A80078D115F4907F8ED0D0070AD5E80540F17C
:1039B800D980606C40F00100606450075BD5002935
:1039C8006CD1900770D5100700F1C980616C00298F
:1039D80086D0910609D5AA0607D594F84220222A4E
:1039E80003D12046FFF700FF23685A69616C02F093
:1039F800400201F0080152EA01055CD12046FFF7B8
:103A08002DFE65646CE790F84230222B7FF468AF96
:103A180003B0BDE83040FFF7E7BE94F84120212A03
:103A28007FF45EAFA168226AB1F5805F00F0D980AB
:103A3800511C216212785A60E28C013A92B2E284F7
:103A4800002A7FF44DAFDA6822F08002DA60DA6883
:103A580042F04002DA6043E72021DA68204622F08B
:103A68004002DA6084F84110FFF7C4FD38E7E80542
:103A78009FD4500712D4900716D50029A3D0616CA3
:103A880041F0040161641107A0D5616C41F008019F
:103A980061649BE7D007EAD450075BD5606C40F0BF
:103AA800020060649007EAD410078FD505F0200063
:103AB80008438BD0E9E703F10C0252E8002F22F407
:103AC800907203F10C0040E800210029F3D103F1C2
:103AD800140252E8002F22F0010203F1140040E81A
:103AE80000210029F3D1226B012A22D000222021B3
:103AF80084F8421022635A69550627D503F1140247
:103B080052E8002F22F0400203F1140040E800219F
:103B18000029F3D1E06BC8B1374B4363FEF764F873
:103B280000283FF4DDAEE06B436B03B0BDE83040E6
:103B3800184703F10C0252E8002F22F0100203F19B
:103B48000C0040E800210029F3D1CFE72046FFF719
:103B580085FDC5E6910792D4110796D436E7A906E4
:103B680093D433E750073FF52CAF84E7E18DE28D1E
:103B7800A08D92B289B2002A3FF4B2AE411A89B23E
:103B880000293FF4ADAE03F10C0252E8002F22F4F5
:103B9800907203F10C0545E800200028F3D103F1E9
:103BA800140252E8002F22F0010203F1140545E83F
:103BB80000200028F3D1202284F84220206303F15A
:103BC8000C0252E8002F22F0100203F10C0545E820
:103BD80000200028F3D1022320466363FFF7A6FDE7
:103BE8007EE6216900297FF423AF32F8021BC1F376
:103BF8000801596022621FE725370008F0B5002543
:103C08004FF0220E0446456480F842E081628285C6
:103C18001346C06B0A46DFF878C021681D4F1E4E58
:103C280083B00431C0E90AC7C0E90C65FDF776FF27
:103C380023680195196822690191596801910199D0
:103C48005AB103F10C0252E8002F42F4807203F1DA
:103C58000C0040E800210029F3D103F1140252E8D6
:103C6800002F42F0010203F1140040E8002100296E
:103C7800F3D103F1140252E8002F42F0400203F19D
:103C8800140141E800200028F3D103B0F0BD00BFC3
:103C980059370008393700086936000890F842C0DB
:103CA800BCF1200F05D130B401B122B930BC0120DC
:103CB8007047022070470024046330BCFFF79EBFA2
:103CC80038B505460C460E4B1A6813681B06FCD51A
:103CD8000120FDF74BFB00232A0A62F3070365F373
:103CE8000F23220A074962F3174364F31F634B60EB
:103CF800054B08220B600248BDE83840FFF7C6BBF9
:103D080030020020B0050020A55A0582F8B5074604
:103D18000C461646194B1D682B681B06FCD501205E
:103D2800FDF724FB45F6A5228223154D6F712A80E5
:103D38003F0A721D2F71AA70EB70DEB1062306EBE5
:103D4800030C611E5FFA8CFC1846013311F8014F11
:103D5800DBB263452C54F7D1F41D06F10802E4B236
:103D6800D2B2FF26EE542E5505490448BDE8F84066
:103D7800FFF78CBB082207240623F2E73002002055
:103D8800B005002038B504460D46184B1A6813686C
:103D98001B06FCD50120FDF7E9FA012245F6A5200E
:103DA8008421134B1A71AA1852001880D9709A707E
:103DB800ADB1204604EB450102880233120ADA70DD
:103DC80030F8022B88421A71F6D16A1ED2B252001C
:103DD800074906480732BDE83840FFF757BB0522B8
:103DE800BDE8384002490148FFF750BB30020020C7
:103DF800B005002000B5184B1A6813681B06FCD5DF
:103E0800012245F6A52E4FF0840C144B1A718A181E
:103E18005200A3F800E083F803C09A70A1B100EB48
:103E2800410C02880233120ADA7030F8022B60451E
:103E38001A71F6D14A1ED2B25200084906485DF8F6
:103E480004EB0732FFF722BB0522044902485DF85C
:103E580004EBFFF71BBB00BF30020020B0050020B9
:103E680038B505460C461A4B1A6813681B06FCD56C
:103E78000120FDF77BFA174B17492A0A19601A71B6
:103E88005D7134B1013C032C1CD8DFE804F0151334
:103E9800191712490C220B254FF00A0CC3F806100B
:103EA800FF2403F80C405C550A490948BDE838402E
:103EB800FFF7ECBA0A49EDE70A49EBE70A49E9E7EF
:103EC8000A49E7E7082207254FF0060CE8E700BF94
:103ED80030020020B0050020A55A09820001000226
:103EE80000050006000300040009000A0007000896
:103EF80010B504460C4B1A6813681B06FCD5012044
:103F0800FDF734FA4FF0020C084B0949A3FB0434BF
:103F1800084BE4080B604C7181F804C00622BDE828
:103F280010400148FFF7B2BA30020020CDCCCCCC0B
:103F3800B0050020A55A038010B56FF04001002499
:103F48000D4B82B01B68DA6842F01002DA60196023
:103F580001941A6801925B680193019B00F09AFE34
:103F680000F040FD4FF480722146044802B0BDE8DD
:103F7800104000F0E9BF00BF300200208802002096
:103F880070B5814B1A7862BB804D814C2B88218893
:103F98000B4499B21BB2002B20DB282B01DD282310
:103FA800194601202B80FFF78BFEB5F90000FCF7BE
:103FB800B3FB73A3D3E90023FCF732F9FCF79EFCAB
:103FC80040F6FF73014600228B42A8BF0B4671489A
:103FD8001146FDF70DFD0023238070BD13461146E1
:103FE800DFE7012A05D0022A1AD00023684C238073
:103FF80070BD674CB4F90030002B32DD664DB5F961
:104008000010132950DC01EB430109B2142967DCC5
:104018002980142966D0322389B203FB01F139E0E3
:104028005E4D5B4C2988238819440BB2002B89B25A
:1040380062DDB3F5FA7F02DD4FF4FA731946032007
:104048002B80FFF73DFE42F21073B5F90000544A89
:1040580093FBF0F31168013BCB62D360002323800C
:1040680070BDB8D04C4DB5F9002091B2C81E1128CA
:1040780045D801EB430109B2012967DD29801229DE
:10408800C9D1484902220520FFF740FE322329887A
:1040980003FB01F1B1F57A7F1DD2022089B2FFF747
:1040A8000FFE0023238070BDB1F5FA6F10DA03EB21
:1040B800830301EB830109B23B4EB1F5FA6F337804
:1040C80029802FDD4FF4FA622A8073B3374902E062
:1040D800322303FB01F1364BA3FB01318909DCE7ED
:1040E80014232B80334902220520FFF70FFE3223C9
:1040F800298803FB01F1CDE7012319469FE7142A1C
:1041080020DD03EB830301EB830109B21329298026
:1041180020DC1422244E2A803378012B20D04FF43F
:104128007A71D8E7002B7FF474AF23490522102059
:10413800FFF7ECFD0120FDF719F90123B5F900108F
:10414800337066E7322303FB01F1A3E702236421FE
:104158002B80A2E71429BBD1134E3378012BDED173
:10416800164905221020FFF7D1FD0120FDF7FEF8C2
:104178000023B5F90010337081E700BFAFF300806A
:104188002F9FF7F279DF5940840200208202002035
:1041980080020020B00000200E0000200C0000204B
:1041A8000C0100201C5000087E020020A08601009F
:1041B800D34D621010500008085000081450000831
:1041C80038B500F03FFC002833D00138152830D826
:1041D800DFE800F04C2F2F5F2F2F0B2F2F70782F39
:1041E8002F2F2F2F2F2F802F2F307B4CB4F90030FB
:1041F800632B40F39E80B3F5FA7FBCBF32331BB20A
:104208000320764AD91782FB0323C1EBA30101EBF4
:104218008101490089B22180FFF752FD42F21073F3
:10422800B4F900006E4A93FBF0F31168013BCB62CE
:10423800D36038BD684CB4F90030642B00F3948027
:10424800012BC8BF0A3B654AC8BF1BB2D91782FBFE
:104258000323C1EBA30101EB810149000BB289B231
:104268000BB90123194603202380D5E76420FFF703
:104278003FFE5C4B202019780131C9B202298CBF5E
:1042880000220A461A7088BF1146BDE83840FFF779
:10429800E7BD554CB4F9001013294DDC023109B2C1
:1042A800218014293DD1514902220520FFF72EFD16
:1042B800218837E00022BDE838404FF400414C48DF
:1042C800FDF7C4BF0122BDE838404FF4004148481B
:1042D800FDF7BCBF444CB4F9003099B2CA1E112A8C
:1042E8001AD9142B1EDDA1F1C80319B221809BB283
:1042F80000294CD114223F4D22802B78012B5DD010
:104308004FF47A713C4BA3FB013189090220BDE8C7
:10431800384089B2FFF7D4BC023909B2218012298A
:104328002ED089B2322303FB01F1B1F57A7FEDD3A8
:10433800E8E70A331BB263E7B1F5FA6F10DA2F4AE0
:1043480001F1C8039BB2A2FB03235B09294D03EBD0
:10435800830303EB830189002A7889B22180E2B1C3
:10436800322303FB01F1CDE7254A323B9BB2A2FB86
:104378000323DB0803EB83035B0099B21BB272E7EC
:10438800204902220520FFF7C1FC2188CAE7142929
:1043980010DD322103FB01F1B4E71B49052210208F
:1043A800FFF7B4FC0120FCF7E1FF0123B4F900108A
:1043B8002B7076E70F4D2B78012BB0D113490522CE
:1043C8001020FFF7A3FC0120FCF7D0FF0023B4F96D
:1043D80000102B70A3E700BF0C000020676666661C
:1043E8000C010020840200200E000020105000085C
:1043F800000801407D020020D34D62101F85EB515B
:10440800CDCCCCCC1C500008085000081450000833
:10441800022800D07047014608B51148FDF710FF83
:1044280028B1BDE808406421022000F049BD00F130
:104438008040042100F58430FDF702FF012804D1F3
:10444800084A138801331380EBE704210448FDF779
:10445800F7FE0028E5D1034A1388013B1380E0E703
:104468000008014080020020322303FB00F0B0F571
:104478007A7F03D3024BA3FB0030800980B27047D8
:10448800D34D621000000000F8B504213848FEF74B
:104498007FFB4FF49671012000F012FD354B1C781C
:1044A8008CBB012234491A70B1F900504FF4807264
:1044B800142D2146314827DC00F046FD00E0013488
:1044C800202CFCD92046FCF727F9064628460F463B
:1044D800FCF722F922A3D3E90023FBF7A1FE00226F
:1044E800274BFBF7CDFF02460B4630463946FCF713
:1044F800DDF920B1234A214B128823F81420013416
:10450800802CDDD126E0F8BD00F01EFD00E001346E
:10451800202CFCD92046FCF7FFF8064628460F4613
:10452800FCF7FAF810A3D3E90023FBF779FE002281
:10453800134BFBF7A5FF02460B4630463946FCF7FE
:10454800B5F920B10F4A0D4B128823F81420013415
:10455800802CDDD17D21BDE8F8400848FFF74ABC32
:104568009A99999999990940FCA9F1D24D62A03F6D
:10457800C40000207F0200200E00002088020020D6
:1045880000004040820200202DE9F843B04C237817
:104598003BB145F6A522AF4B1988914203D00023C1
:1045A8002370BDE8F8839A78062AF8D1DA78832A46
:1045B800F5D1B3F807305BBA9BB2013B072BEED8B5
:1045C800DFE813F0F400B400DF009C008900670006
:1045D80054000800A04E3378012B00F0EF8004212E
:1045E8003020FFF73DFC01229C499D4BB1F900703A
:1045F8001A70142F4FF480724FF00001994800F39D
:10460800668100F0A1FC002500E00135202DFCD9D1
:104618002846FCF781F8804638468946FCF77CF83E
:1046280087A3D3E90023FBF7FBFD00228E4BFBF7A2
:1046380027FF02460B4640464946FCF737F920B1AA
:104648008A4A884B128823F815200135802DDDD140
:104658007D218448FFF796FB6FF0010284480368C8
:104668001A61FEF75DF90123337098E77A4E3378C3
:10467800012B00F0A3807F4D04212846FEF7E6FABF
:10468800764B2A68B3F90030013B9363FFF7FCFED1
:1046980085E7794DB5F90020632A00F3CB800A320B
:1046A80012B203207549D31781FB0212C3EBA20390
:1046B80003EB8303590089B22980FFF701FB42F21B
:1046C8001073B5F900006A4A93FBF0F31168013BD7
:1046D800CB62D36063E7684DB5F90030642B77DDB2
:1046E800674A323B9BB2A2FB0323DB0803EB83033D
:1046F8005B0099B21BB203202B80DEE7574DB5F95A
:104708000010132979DC02310BB22B80142B00F036
:104718000D8132229BB202FB03F1B1F57A7F80F062
:104728008480022089B2FFF7CBFA38E74F4DB5F9FC
:104738000030272BDCBF05331BB2504AD91782FB48
:104748000323C1EB630101EB810189B201202980B8
:10475800FFF7B6FAB5F90000FBF7DEFF3AA3D3E995
:104768000023FBF75DFDFCF7C9F840F6FF7301462F
:1047780000228B42A8BF0B4642481146FDF738F984
:104788000DE7364DB5F9002093B2D91E11297FD80F
:10479800023B9BB2122B2B8000F0C180322202FB1D
:1047A80003F3022099B2FFF78BFAF8E62F4DB5F91B
:1047B8000030002BC1DD053B1BB2BEE72C48FEF7DD
:1047C800E1F80223032130203370FFF749FBE6E6C6
:1047D800012BC8BF0A3B294AC8BF1BB2D91782FBA5
:1047E8000323C1EBA30101EB810149000BB289B29C
:1047F800002B80D1012319467DE7B1F5FA6F11DA54
:10480800642001F1C8039BB2B3FBF0F31E4E03EB27
:10481800830303EB83039900327889B22980002A45
:1048280000F09280322303FB01F1184BA3FB013106
:10483800890976E7B2F5FA7FBCBF323212B230E7A7
:104848009A999999999909402F9FF7F279DF5940D8
:10485800B0090020B0030020100000200E00002046
:104868007F020020880200200000404082020020D1
:104878000C010020C40000200C000020676666665A
:10488800CDCCCCCCB00000207C020020D34D6210EF
:10489800142A10DDC83B1AB22A809BB2002A4DD1D7
:1048A80014232B80384E3778012F5AD0B5F90020C1
:1048B800122A34D093B2322202FB03F3B3F57A7F83
:1048C800FFF46FAF314AA2FB03239B0969E700F0AD
:1048D8003BFB002500E00135202DFCD93846FBF7CD
:1048E8001BFF27A3D3E90023FBF79AFC0022284BE0
:1048F800FBF7C6FD804628468946FBF70DFF0246B2
:104908000B4640464946FBF7EFFF20B1214A224BB0
:10491800128823F815200135802DDDD198E6022272
:1049280005201E49FFF7F2F92B88C4E7022205206B
:104938001B49FFF7EBF9B5F90030EAE6142AB1DDB7
:10494800322202FB03F3BDE7052210201549FFF7C9
:10495800DDF90120FCF70AFD0122B5F900303270BB
:10496800D4E6052210201049FFF7D0F93846FCF7A5
:10497800FDFC0023B5F90020337099E7AFF3008000
:10498800FCA9F1D24D62A03F7C020020D34D6210F9
:104998000000404082020020880200201C500008CD
:1049A8001050000808500008145000080368B3F1BC
:1049B800804F00D0704710B5074C04212046FEF701
:1049C80045F9064B2268B3F90030BDE81040013BB9
:1049D8009363FFF759BD00BFC40000200E000020FC
:1049E80000F048B800220221144B15489A60428111
:1049F800027319711A7319759A611A7783F824105A
:104A08009A6283F82C2083F834109A6383F83C2048
:104A180083F844109A6483F84C2083F854109A65FC
:104A280083F85C2083F864109A6683F86C2083F816
:104A380074109A6783F87C20704700BFC40900206F
:104A4800B4090020074A917AD37A8B4207D04B1CCD
:104A5800DBB20A2B28BF0023505C937270470020FA
:104A6800704700BFB4090020014BDA7A9A72704788
:104A7800B4090020F0B50122002405253C483D4B2F
:104A88000AE01D71DC801C730332D2B2192A00F1CE
:104A9800080003F1100336D00168B0F804C0896833
:104AA80090F806E01CEA010F14BF4FF0010C4FF01C
:104AB800000CE645197905D00529E2D831B101394C
:104AC8001971DFE7042919D81D71DDE793F80AC0C9
:104AD800BCF1010FD6D1284E02F1010E96F80BC099
:104AE800997206F80CE00CF1010C5FFA8CFCBCF131
:104AF800090F94BF86F80BC0F172C3E7092903D8E0
:104B080001311971C0E7F0BD9E7A56B901211A4FDB
:104B18009972F97A7A540131C9B2092994BFF972A4
:104B2800FE7219890029AFD0DE88B1420DD8DE7A2D
:104B3800002EA9D0197B0131C9B28E4216D80021A6
:104B480019730D49CE7A8A5508E00136B6B2B142DA
:104B5800DE8099D10849971CCE7A8F550136F6B276
:104B6800092ECE7290D90026CE728DE719738BE785
:104B780020500008C4090020B4090020F8B5FFF748
:104B8800DBF93748FEF7BEFC4FF40072354934486C
:104B9800FFF784F800213448FCF7F6FE1422334965
:104BA8003348FCF7DDFD40F6C410FCF7DFFB0222BA
:104BB80005203049FFF7AAF82F4B20201978FFF776
:104BC8004FF903213020FFF74BF92C4B01201988AE
:104BD800FFF776F82A4B00271888FFF745FC0146AF
:104BE8000220FFF76DF8274B03201988FFF768F8B4
:104BF8007D212548FFF7C6F84FF4FA71384600F0D2
:104C080077F9224EFFF730FF214D1F4C0DE00120B0
:104C180000F088F9C0B9022000F084F908B1FFF764
:104C2800AFF9FFF7CDFAFFF7AFFC002000F07AF9F3
:104C38000028ECD028464FF48051FDF70BFB0120EB
:104C480000F070F90028E6D04FF480720021204669
:104C580000F07AF97D212046FFF794F83770DAE7FB
:104C680030020020B0070020B00000208803002098
:104C7800800000201C5000088402002082020020CE
:104C88000E0000200C000020880200207F02002077
:104C9800000C01400023284A2849536028489360A3
:104CA800537013701361536153731373D361136299
:104CB800537613769362D36282F8253082F82430D3
:104CC8005363936382F8313082F83030136453644D
:104CD80082F83D3082F83C30D364136582F849305D
:104CE80082F848309365D36582F8553082F854309D
:104CF800536609689366A0FB010189090139B1F17E
:104D0800807F82F8613082F860301367536782F8D9
:104D18006D3082F86C300DD24FF0E0224FF0F00C7D
:104D2800072010B4074C516184F823C010BC93616C
:104D380010617047FEE700BF4C0A00200000002009
:104D4800D34D621000ED00E0584B1A6832B11A6872
:104D5800013A1A6012B90122554B1A70554B5A681C
:104D680052B15A68013A5A6032B901225A701A7817
:104D7800012A04BF9A685A601A6952B11A69013A3D
:104D88001A6132B901225A731A7B012A04BF5A697F
:104D98001A61DA6952B1DA69013ADA6132B9012283
:104DA8005A761A7E012A04BF1A6ADA619A6A62B1CF
:104DB8009A6A013A9A6242B9012283F8252093F847
:104DC8002420012A04BFDA6A9A625A6B62B15A6BCC
:104DD800013A5A6342B9012283F8312093F830200E
:104DE800012A04BF9A6B5A631A6C62B11A6C013AB1
:104DF8001A6442B9012283F83D2093F83C20012A25
:104E080004BF5A6C1A64DA6C62B1DA6C013ADA647B
:104E180042B9012283F8492093F84820012A04BFA7
:104E28001A6DDA649A6D62B19A6D013A9A6542B95F
:104E3800012283F8552093F85420012A04BFDA6D23
:104E48009A655A6E62B15A6E013A5A6642B901229F
:104E580083F8612093F86020012A04BF9A6E5A668D
:104E68001A6F62B11A6F013A1A6742B9012283F8C0
:104E78006D2093F86C20012A04BF5A6F1A676FF0EF
:104E880000410D4B1A6801321A601A688A4204BF41
:104E980000221A60094A13780133DBB2092B01D8C2
:104EA8001370704700231370FFF79ABDC80A0020DB
:104EB800C40A00204C0A0020480A0020440A0020A6
:104EC800092812D810B4012383F310880023074C53
:104ED80000EB400004EB8002800051609160537049
:104EE800235483F3108810BC7047FEE74C0A002057
:104EF800092813D830B54FF0010E8EF31088002220
:104F0800074D00EB400005EB800384005960996071
:104F18005A7005F804E082F3108830BDFEE700BF40
:104F28004C0A0020092808D8064B00EB400003EB88
:104F380080035A78012AD0B201D00020704700229D
:104F48005A7070474C0A002003460244934200D12D
:104F5800704703F8011BF9E770B500260C4D0D4C9E
:104F6800641BA410A64209D100F028F800260A4DB7
:104F78000A4C641BA410A64205D170BD55F8043B29
:104F880098470136EEE755F8043B98470136F2E7B3
:104F98006050000860500008605000086450000825
:104FA8000A44914200F1FF3300D1704710B511F85F
:104FB800014B914203F8014FF9D110BDF8B500BF7C
:104FC800F8BC08BC9E467047F8B500BFF8BC08BCE2
:044FD8009E4670473A
:104FDC0000000000010203040000000000000000BB
:104FEC00010203040607080901020000020304057C
:104FFC00060708090A0B0C0D0E0F10102035307522
:10500C0073000000757300003530306E73000000C3
:10501C006E73000000080140080001000008014008
:10502C002000010000080140400001000010014078
:10503C00200001000010014000010100001001409F
:10504C0000020100000C014001000100000C0140B5
:04505C00020001004D
:045060000D02000835
:04506400E901000856
:105068000024F4000100000010000000010002000C
:045078000200000032
:040000050800129944
:00000001FF
